:100000000C9401010C941E010C941E010C941E0111
:100010000C941E010C941E010C941E010C941E01E4
:100020000C941E010C941E010C941E010C941E01D4
:100030000C941E010C94870F0C94BA0F0C94A80E0C
:100040000C94540F0C94EE0E0C94210F0C941E0182
:100050000C94750E0C941E010C941E010C941C0E35
:100060000C941E010C94D3090C941E010C942709C6
:100070000C941E010C941E020C941E010C941E0183
:100080000C941E010C941E010C941E010C941E0174
:100090000C94FE090C941E010C9452090C941E0140
:1000A0000C941E010C941E010C941E010C941E0154
:1000B0000C941E010C941E010C941E010C941E0144
:1000C0000C941E010C941E010C941E010C94290A20
:1000D0000C941E010C947D090C94540A0C941E017E
:1000E0000C94A80900000100080040000001000471
:1000F0000000010008002000400080000001000412
:10010000303132333435363738394142434445464D
:10011000004C5F53656E736F723D25642C204C5FFD
:10012000776865656C3D256425642C20525F5365B6
:100130006E736F723D25642C20525F776865656C25
:100140003D256425640D0A0020706F7274002070D4
:100150006F72740020706F72740020706F72740080
:1001600020330020320020310020300020330020D6
:100170003200203000383A256420393A2564203195
:10018000303A25642031313A25642031323A2564F1
:100190002031333A25642031343A25642031353A10
:1001A0002564200D0A00303A256420313A25642068
:1001B000323A256420333A256420343A25642035C8
:1001C0003A256420363A256420373A2564200D0A02
:1001D00000496E697469616C697A6174696F6E2037
:1001E000436F6D706C657465200D0A002E000D0A5A
:1001F00053797374656D205761726D696E67205510
:10020000700011241FBECFEFD1E2DEBFCDBF12E0E0
:10021000A0E0B2E0E6E8FBE302C005900D92A6394B
:10022000B107D9F715E0A6E9B2E001C01D92AF34DD
:10023000B107E1F70E94BC1C0C94C11D0C94000096
:10024000DF93CF93CDB7DEB7AAE7B0E0EAE7F0E0FF
:10025000808180688C93AAE7B0E0EAE7F0E08081D3
:100260008F7D8C9386E00E94610181E00E94750180
:10027000ACE7B0E0ECE7F0E080818F7D8C93AAE7FB
:10028000B0E0EAE7F0E0808188608C931092F2049D
:100290007894CF91DF910895DF93CF93CDB7DEB7F8
:1002A000AAE7B0E0EAE7F0E08081877F8C93AAE7D5
:1002B000B0E0EAE7F0E080818F778C93CF91DF9117
:1002C0000895DF93CF930F92CDB7DEB78983AAE766
:1002D000B0E0EAE7F0E08081982F987F8981892B50
:1002E0008C930F90CF91DF910895DF93CF930F926E
:1002F000CDB7DEB78983ACE7B0E0ECE7F0E0808112
:10030000282F2F738981882F90E000249695879558
:100310000794969587950794982F802D822B8C9320
:100320000F90CF91DF910895DF93CF930F92CDB7C8
:10033000DEB78983ACE7B0E0ECE7F0E08081982F8E
:10034000907E89818F71892B8C930F90CF91DF9153
:100350000895DF93CF93CDB7DEB7AAE7B0E0EAE721
:10036000F0E0808180618C93AAE7B0E0EAE7F0E0FA
:10037000808180648C93CF91DF910895DF93CF9338
:10038000CDB7DEB7EAE7F0E080818074CF91DF91EE
:100390000895DF93CF930F92CDB7DEB78983109284
:1003A000F2048981883040F0ABE7B0E0EBE7F0E0A1
:1003B000808188608C9307C0ABE7B0E0EBE7F0E0AA
:1003C0008081877F8C93ACE7B0E0ECE7F0E0808140
:1003D000982F987F89818770892B8C93AAE7B0E04A
:1003E000EAE7F0E0808180618C93AAE7B0E0EAE779
:1003F000F0E0808180648C93EAE7F0E08081882FD0
:1004000090E0807490700097B9F7E8E7F0E08081A1
:1004100091810F90CF91DF910895DF93CF930F9249
:10042000CDB7DEB7898389810E94C90196958795EA
:10043000969587950F90CF91DF9108951F920F9217
:100440000FB60F9211248F93DF93CF93CDB7DEB702
:100450008FEF8093F204CF91DF918F910F900FBEB9
:100460000F901F901895DF93CF93CDB7DEB72797E6
:100470000FB6F894DEBF0FBECDBF9B838A837D830A
:100480006C835F834E83EFE5F0E080818983F8948D
:10049000EA81FB818C819D8191838083EA81FB814C
:1004A0008E819F8193838283EA81FB8117821682EA
:1004B000EA81FB8115821482EFE5F0E08981808377
:1004C00027960FB6F894DEBF0FBECDBFCF91DF9158
:1004D0000895DF93CF9300D000D0CDB7DEB79C83D3
:1004E0008B831A82EFE5F0E080818983F894EB81B9
:1004F000FC81848195810097D1F1EB81FC81208181
:100500003181EB81FC8186819781F901E80FF91F28
:1005100080818A83EB81FC81868197810196EB81C2
:10052000FC8197838683EB81FC8126813781EB8177
:10053000FC81828193812817390780F0EB81FC814F
:1005400026813781EB81FC8182819381A901481B3F
:10055000590BCA01EB81FC8197838683EB81FC8177
:10056000848195810197EB81FC8195838483EFE5FC
:10057000F0E0898180838A810F900F900F900F9017
:10058000CF91DF910895DF93CF9300D000D00F92E9
:10059000CDB7DEB79B838A837D836C83EFE5F0E084
:1005A00080818983F894EA81FB81248135818C8163
:1005B0009D8182179307B0F5EA81FB8126813781FF
:1005C0008C819D81820F931FEA81FB8197838683B3
:1005D000EA81FB8126813781EA81FB8182819381D7
:1005E0002817390780F0EA81FB8126813781EA816B
:1005F000FB8182819381A901481B590BCA01EA81C1
:10060000FB8197838683EA81FB81248135818C81FC
:100610009D81A901481B590BCA01EA81FB81958381
:10062000848304C0EA81FB8115821482EFE5F0E047
:10063000898180830F900F900F900F900F90CF9132
:10064000DF9108950F931F93DF93CF9300D000D0D5
:1006500000D0CDB7DEB79C838B837E836D83EFE5BF
:10066000F0E080818A83F894EB81FC810081118124
:10067000EB81FC81268137818D819E81820F931FC2
:10068000EB81FC8122813381B9010E945D1DF8015B
:10069000E80FF91F80818983EFE5F0E08A8180838C
:1006A000898126960FB6F894DEBF0FBECDBFCF91DD
:1006B000DF911F910F9108950F931F93DF93CF93B5
:1006C00000D000D00F92CDB7DEB79B838A836C83B6
:1006D000EFE5F0E080818983F894EA81FB81248151
:1006E0003581EA81FB81828193812817390750F592
:1006F000EA81FB8100811181EA81FB8126813781BA
:10070000EA81FB8184819581820F931FEA81FB81BD
:1007100022813381B9010E945D1DF801E80FF91FA4
:100720008C818083EA81FB81848195810196EA81B5
:10073000FB8195838483EFE5F0E0898180838FEFEF
:100740008D8305C0EFE5F0E0898180831D828D8176
:100750000F900F900F900F900F90CF91DF911F91FE
:100760000F910895DF93CF9300D000D00F92CDB7B3
:10077000DEB79D838C83EFE5F0E080818B83F89476
:10078000EC81FD8122813381EC81FD818481958121
:10079000A901481B590BCA019A838983EFE5F0E050
:1007A0008B81808389819A810F900F900F900F9099
:1007B0000F90CF91DF910895DF93CF9300D00F92E8
:1007C000CDB7DEB79B838A83EFE5F0E08081898334
:1007D000F894EA81FB8115821482EFE5F0E08981CB
:1007E00080830F900F900F90CF91DF910895DF934A
:1007F000CF93CDB7DEB70E9406040E9428040E9462
:100800004A040E946C04CF91DF910895DF93CF9347
:10081000CDB7DEB70E948E041092D7041092D60492
:10082000E1ECF0E088ED808340E855E260E070E0C4
:1008300080E00E9418058FEF8093F3041092170553
:1008400010923C0510923B057894CF91DF9108956A
:10085000DF93CF93CDB7DEB70E94A9041092D904DD
:100860001092D804E9ECF0E088ED808340E855E28E
:1008700060E070E081E00E9418058FEF8093F4043F
:100880001092180510923E0510923D057894CF9174
:10089000DF910895DF93CF93CDB7DEB70E94C404F4
:1008A0001092DB041092DA04E1EDF0E088ED808331
:1008B00040E855E260E070E082E00E9418058FEFAA
:1008C0008093F504109219051092400510923F058F
:1008D0007894CF91DF910895DF93CF93CDB7DEB7B2
:1008E0000E94DF041092DD041092DC04E1E3F1E0E9
:1008F00088ED808340E855E260E070E083E00E948C
:1009000018058FEF8093F60410921A051092420595
:10091000109241057894CF91DF910895DF93CF93A2
:10092000CDB7DEB786E992E027EF34E040E850E04B
:10093000BC01C9010E94330286E193E02BE135E05E
:1009400040E150E0BC01C9010E943302CF91DF9128
:100950000895DF93CF93CDB7DEB786E293E02FEF14
:1009600034E040E850E0BC01C9010E94330286EA4D
:1009700093E023E235E040E150E0BC01C9010E9470
:100980003302CF91DF910895DF93CF93CDB7DEB7D8
:1009900086EB93E027E035E040E850E0BC01C90178
:1009A0000E94330286E394E02BE235E040E150E020
:1009B000BC01C9010E943302CF91DF910895DF93FA
:1009C000CF93CDB7DEB786E494E02FE035E040E882
:1009D00050E0BC01C9010E94330286EC94E023E39D
:1009E00035E040E150E0BC01C9010E943302CF91E3
:1009F000DF910895DF93CF9300D00F92CDB7DEB78C
:100A000089837B836A838981843060F48981882F1C
:100A100090E0880F991FFC01EA52FB4F8A819B816D
:100A2000918380830F900F900F90CF91DF91089565
:100A3000EF92FF920F931F93DF93CF93CDB7DEB763
:100A400027970FB6F894DEBF0FBECDBF8B834C83C4
:100A50005D836E837F838C819D81AE81BF81805851
:100A60009B47A14EBF4F880F991FAA1FBB1F880F1E
:100A7000991FAA1FBB1F880F991FAA1FBB1F7C01AC
:100A80008D018C819D81AE81BF81880F991FAA1F26
:100A9000BB1F880F991FAA1FBB1F880F991FAA1F72
:100AA000BB1F880F991FAA1FBB1F9C01AD01C80166
:100AB000B7010E94841DDA01C90101979A838983D5
:100AC0008B81833061F4E4E3F1E089818083E5E3A5
:100AD000F1E089819A81892F9927808329C08B81B0
:100AE000823061F4E4EDF0E089818083E5EDF0E0AF
:100AF00089819A81892F992780831AC08B818130BF
:100B000061F4ECECF0E089818083EDECF0E0898128
:100B10009A81892F992780830BC0E4ECF0E08981CA
:100B20008083E5ECF0E089819A81892F9927808381
:100B300027960FB6F894DEBF0FBECDBFCF91DF91E1
:100B40001F910F91FF90EF900895DF93CF930F9235
:100B5000CDB7DEB789838981882F90E0880F991FF0
:100B6000880F991F880F991F89509B4F0F90CF9125
:100B7000DF910895DF93CF930F92CDB7DEB78983CE
:100B80008981882F90E0880F991F880F991F880FFF
:100B9000991F855E9A4F0F90CF91DF910895DF9353
:100BA000CF9300D0CDB7DEB789836A838981833044
:100BB00071F4E0E3F1E08081882F90E08072907022
:100BC0000097B9F3E6E3F1E08A8180832FC0898141
:100BD000823071F4E0EDF0E08081882F90E0807247
:100BE00090700097B9F3E6EDF0E08A8180831EC033
:100BF0008981813071F4E8ECF0E08081882F90E009
:100C0000807290700097B9F3EEECF0E08A818083F7
:100C10000DC0E0ECF0E08081882F90E08072907051
:100C20000097B9F3E6ECF0E08A8180838981882F10
:100C300090E0FC01ED50FB4F10820F900F90CF9190
:100C4000DF910895DF93CF930F92CDB7DEB78983FD
:100C5000698180E00E94CF050F90CF91DF910895C8
:100C6000DF93CF930F92CDB7DEB78983698181E09F
:100C70000E94CF050F90CF91DF910895DF93CF931E
:100C80000F92CDB7DEB78983698182E00E94CF05DC
:100C90000F90CF91DF910895DF93CF930F92CDB74F
:100CA000DEB78983698183E00E94CF050F90CF91E1
:100CB000DF910895DF93CF9300D00F92CDB7DEB7C9
:100CC000CE010196BC0180E00E94DA06882331F053
:100CD0008981282F30E03B832A8304C08FEF9FEF68
:100CE0009B838A838A819B810F900F900F90CF9175
:100CF000DF910895DF93CF9300D00F92CDB7DEB789
:100D0000CE010196BC0181E00E94DA06882331F011
:100D10008981282F30E03B832A8304C08FEF9FEF27
:100D20009B838A838A819B810F900F900F90CF9134
:100D3000DF910895DF93CF9300D00F92CDB7DEB748
:100D4000CE010196BC0182E00E94DA06882331F0D0
:100D50008981282F30E03B832A8304C08FEF9FEFE7
:100D60009B838A838A819B810F900F900F90CF91F4
:100D7000DF910895DF93CF9300D00F92CDB7DEB708
:100D8000CE010196BC0183E00E94DA06882331F08F
:100D90008981282F30E03B832A8304C08FEF9FEFA7
:100DA0009B838A838A819B810F900F900F90CF91B4
:100DB000DF910895DF93CF9300D000D0CDB7DEB799
:100DC00089837B836A838981882F90E0880F991FAC
:100DD000880F991F0196880F991FFC01E950FB4F5E
:100DE00080819181009731F18981882F90E0880F6F
:100DF000991F0196880F991F880F991FFC01E950D0
:100E0000FB4F80819181009799F08981882F90E034
:100E1000880F991F880F991F880F991F89509B4F22
:100E20000E946902EA81FB8180838FEF8C8303C07B
:100E30001C8201C01C828C810F900F900F900F902C
:100E4000CF91DF910895DF93CF930F92CDB7DEB7A7
:100E500089838981882F90E0880F991F880F991FB7
:100E6000880F991F89509B4F0E94DC030F90CF91F0
:100E7000DF910895DF93CF9300D0CDB7DEB789839C
:100E80008981882F90E0880F991F0196880F991FFC
:100E9000880F991FFC01E950FB4F808191811A82D4
:100EA000009711F481E08A838A810F900F90CF918F
:100EB000DF910895DF93CF9300D0CDB7DEB789835C
:100EC0006A838981882F90E0880F991F880F991F66
:100ED000880F991F855E9A4F6A810E945C030F906C
:100EE0000F90CF91DF910895DF93CF930F92CDB7FD
:100EF000DEB78983698180E00E945A070F90CF9105
:100F0000DF910895DF93CF930F92CDB7DEB789833A
:100F1000698181E00E945A070F90CF91DF91089577
:100F2000DF93CF930F92CDB7DEB78983698182E0DB
:100F30000E945A070F90CF91DF910895DF93CF93CE
:100F40000F92CDB7DEB78983698183E00E945A078B
:100F50000F90CF91DF910895DF93CF930F92CDB78C
:100F6000DEB789838981882F90E0FC01E95EFA4F22
:100F70008FEF80838981882F90E0880F991F880FD9
:100F8000991F880F991F855E9A4F0E946902682FEA
:100F900089810E94CF050F90CF91DF910895DF9353
:100FA000CF93CDB7DEB729970FB6F894DEBF0FBE4B
:100FB000CDBF89837B836A835D834C838981882F3E
:100FC00090E0880F991F0196880F991F880F991F2D
:100FD000FC01E55EFA4F208131818C819D81280FD3
:100FE000391F8981882F90E0880F991F880F991FDA
:100FF0000196880F991FFC01E55EFA4F808191816F
:101000002817390708F043C08C819D81009709F4A7
:101010003EC0EA81FB81208128878A819B810196DD
:101020009B838A831F821E821BC0EA81FB812081F1
:101030008A819B8101969B838A838981882F90E096
:10104000880F991F880F991F880F991F855E9A4FE7
:10105000622F0E945C038E819F8101969F838E8305
:101060008C819D8101972E813F8128173907E8F2F5
:101070008981882F90E0FC01E95EFA4F8FEF808331
:10108000688589810E94CF053FEF398701C01986A5
:10109000898529960FB6F894DEBF0FBECDBFCF91DC
:1010A000DF9108950F931F93DF93CF930F92CDB7E6
:1010B000DEB789838981882F90E0FC01E95EFA4FD1
:1010C0008081882309F44EC08981882F90E0880FA1
:1010D000991F0196880F991F880F991FFC01E55EE3
:1010E000FA4F80819181009769F18981833049F4B9
:1010F00006E311E083E395E00E946902F801808332
:1011000039C08981823049F406ED10E08BE295E028
:101110000E946902F80180832DC08981813049F4E1
:101120000EEC10E083E295E00E946902F8018083F2
:1011300021C006EC10E08BE195E00E946902F80105
:10114000808318C08981882F90E0FC01E95EFA4F06
:1011500010828981882F90E0FC01ED50FB4F8FEFCA
:10116000808308C08981882F90E0FC01ED50FB4FFF
:101170008FEF80830F90CF91DF911F910F91089592
:10118000DF93CF9300D0CDB7DEB78A838A818330D7
:1011900029F4E6E3F1E08081898314C08A818230FA
:1011A00029F4E6EDF0E0808189830CC08A818130EA
:1011B00029F4EEECF0E08081898304C0E6ECF0E0F5
:1011C000808189838A81882F90E0880F991FFC0194
:1011D000EA52FB4F80819181009771F08A81882FBC
:1011E00090E0880F991FFC01EA52FB4F0190F081BB
:1011F000E02D8981099526C08A81882F90E0880F8B
:10120000991F880F991F880F991F89509B4F6981DB
:101210000E945C038823B1F48A81282F30E0C90141
:10122000880F991FFC01E55CFA4F80819181AC0128
:101230004F5F5F4FC901880F991FFC01E55CFA4FB2
:10124000518340830F900F90CF91DF9108951F92AB
:101250000F920FB60F9211242F933F934F935F93EA
:101260006F937F938F939F93AF93BF93EF93FF936E
:10127000DF93CF93CDB7DEB780E00E945208CF91C5
:10128000DF91FF91EF91BF91AF919F918F917F91EE
:101290006F915F914F913F912F910F900FBE0F90E3
:1012A0001F9018951F920F920FB60F9211242F9333
:1012B0003F934F935F936F937F938F939F93AF93DE
:1012C000BF93EF93FF93DF93CF93CDB7DEB781E06A
:1012D0000E945208CF91DF91FF91EF91BF91AF91A2
:1012E0009F918F917F916F915F914F913F912F913E
:1012F0000F900FBE0F901F9018951F920F920FB670
:101300000F9211242F933F934F935F936F937F938B
:101310008F939F93AF93BF93EF93FF93DF93CF93FD
:10132000CDB7DEB782E00E945208CF91DF91FF91E6
:10133000EF91BF91AF919F918F917F916F915F914D
:101340004F913F912F910F900FBE0F901F901895C6
:101350001F920F920FB60F9211242F933F934F932A
:101360005F936F937F938F939F93AF93BF93EF930D
:10137000FF93DF93CF93CDB7DEB783E00E9452088F
:10138000CF91DF91FF91EF91BF91AF919F918F919D
:101390007F916F915F914F913F912F910F900FBE71
:1013A0000F901F9018951F920F920FB60F92112455
:1013B0002F933F934F935F936F937F938F939F935D
:1013C000AF93BF93EF93FF93DF93CF93CDB7DEB788
:1013D00080E00E94C008CF91DF91FF91EF91BF9113
:1013E000AF919F918F917F916F915F914F913F91BD
:1013F0002F910F900FBE0F901F9018951F920F9274
:101400000FB60F9211242F933F934F935F936F93D7
:101410007F938F939F93AF93BF93EF93FF93DF934C
:10142000CF93CDB7DEB781E00E94C008CF91DF91A6
:10143000FF91EF91BF91AF919F918F917F916F91AC
:101440005F914F913F912F910F900FBE0F901F9082
:1014500018951F920F920FB60F9211242F933F935E
:101460004F935F936F937F938F939F93AF93BF93AC
:10147000EF93FF93DF93CF93CDB7DEB782E00E9467
:10148000C008CF91DF91FF91EF91BF91AF919F91F4
:101490008F917F916F915F914F913F912F910F901D
:1014A0000FBE0F901F9018951F920F920FB60F92BC
:1014B00011242F933F934F935F936F937F938F9359
:1014C0009F93AF93BF93EF93FF93DF93CF93CDB7EA
:1014D000DEB783E00E94C008CF91DF91FF91EF91CA
:1014E000BF91AF919F918F917F916F915F914F913C
:1014F0003F912F910F900FBE0F901F901895DF9383
:10150000CF9300D000D000D0CDB7DEB79C838B83C3
:101510008B819C81039625E030E0B9010E945D1D1E
:10152000CB01CC01A0E0B0E0880F991FAA1FBB1F20
:10153000880F991FAA1FBB1F880F991FAA1FBB1FC7
:10154000880F991FAA1FBB1F9A8389831E821D8241
:1015500006C02D813E812F5F3F4F3E832D838981C1
:101560009A812D813E812817390798F326960FB668
:10157000F894DEBF0FBECDBFCF91DF910895DF930A
:10158000CF930F92CDB7DEB7198206C089810E9432
:10159000E40B89818F5F898389818730B8F30E944A
:1015A000DA0A0E94F00A0E94050B78940F90CF91FE
:1015B000DF910895DF93CF93CDB7DEB785E00E942A
:1015C0001B0BE6E4F0E01082AEE6B0E0EEE6F0E001
:1015D000808181608C930E94D10CCF91DF9108951E
:1015E000DF93CF93CDB7DEB783E00E942F0BE4E803
:1015F000F0E011821082AFE6B0E0EFE6F0E080812B
:1016000081608C93CF91DF910895DF93CF93CDB715
:10161000DEB784E00E94430BE2EBF0E01082A0E72B
:10162000B0E0E0E7F0E0808181608C930E94F10CF3
:10163000CF91DF910895DF93CF930F92CDB7DEB7AF
:101640008983A5E4B0E0E5E4F0E08081982F987FFD
:101650008981892B8C930F90CF91DF910895DF932F
:10166000CF930F92CDB7DEB78983A1E8B0E0E1E870
:10167000F0E08081982F987F8981892B8C930F903F
:10168000CF91DF910895DF93CF930F92CDB7DEB75F
:101690008983A1EBB0E0E1EBF0E08081982F987FA7
:1016A0008981892B8C930F90CF91DF910895DF93DF
:1016B000CF9300D000D0CDB7DEB7E5E4F0E0808175
:1016C000882F90E087709070880F991F8C519F4FE2
:1016D0009C838B838B819C81FC01859194919A835F
:1016E0008983FC83EB8389819A810F900F900F90FF
:1016F0000F90CF91DF910895DF93CF9300D000D06A
:10170000CDB7DEB7E1E8F0E08081882F90E0877008
:101710009070880F991F8C519F4F9C838B838B8176
:101720009C81FC01859194919A838983FC83EB834E
:1017300089819A810F900F900F900F90CF91DF9138
:101740000895DF93CF9300D000D0CDB7DEB7E1EBA3
:10175000F0E08081882F90E087709070880F991F4B
:1017600080519F4F9C838B838B819C81FC01859151
:1017700094919A838983FC83EB8389819A810F906A
:101780000F900F900F90CF91DF910895DF93CF933B
:1017900000D00F92CDB7DEB789837B836A838981BE
:1017A000873060F48981882F90E0880F991FFC01B1
:1017B000E252FB4F8A819B81918380830F900F902F
:1017C0000F90CF91DF910895DF93CF930F92CDB714
:1017D000DEB789838981873050F48981882F90E032
:1017E000880F991FFC01E252FB4F118210820F906B
:1017F000CF91DF910895EF92FF920F931F93DF93A4
:10180000CF93CDB7DEB72F970FB6F894DEBF0FBEDC
:10181000CDBF9B878A87E6E4F0E0808189871092BC
:101820004705109248051092490510924A050E94FA
:10183000570B9C0140E050E080E094E2A4EFB0E060
:10184000BC01CD010E94A61DDA01C9018D839E83D2
:10185000AF83B8878D819E81AF81B885893B2DE8A4
:10186000920726E0A20720E0B20720F58A859B8533
:10187000A7E281319A07F0F48A859B85CC01A0E02C
:10188000B0E02D813E814F815885BC01CD010E9481
:101890003E1DDC01CB0128EE33E040E050E0BC010E
:1018A000CD010E94841DDA01C90189839A83AB832B
:1018B000BC833EC08A859B857C0100E010E08D8161
:1018C0009E81AF81B88528EE33E040E050E0BC0156
:1018D000CD010E94841DDA01C9019C01AD01C8013E
:1018E000B7010E943E1DDC01CB0189839A83AB8343
:1018F000BC831EC08091470590914805A091490581
:10190000B0914A05A3E5B0E0E3E5F0E08081817F96
:101910008C93A3E5B0E0E3E5F0E0808181608C93F7
:101920008895A3E5B0E0E3E5F0E080818E7F8C93BD
:101930008091470590914805A0914905B0914A05CD
:101940002227382F492F5A2FE6E4F0E08081882F94
:1019500090E0A0E0B0E079018A01E82AF92A0A2B98
:101960001B2B8985282F30E040E050E089819A8147
:10197000AB81BC81820F931FA41FB51FE816F90627
:101980000A071B0708F4B6CF2F960FB6F894DEBFF0
:101990000FBECDBFCF91DF911F910F91FF90EF90C0
:1019A0000895DF93CF93CDB7DEB710924305109221
:1019B00044051092450510924605CF91DF91089598
:1019C000DF93CF93CDB7DEB7809143059091440567
:1019D000A0914505B0914605BC01CD01CF91DF91A5
:1019E0000895DF93CF93CDB7DEB710924B051092D9
:1019F0004C0510924D0510924E05CF91DF91089540
:101A0000DF93CF93CDB7DEB780914B0590914C0516
:101A1000A0914D05B0914E05BC01CD01CF91DF9154
:101A20000895DF93CF930F92CDB7DEB78983898175
:101A3000893079F4A0E8B0E0E0E8F0E080818260ED
:101A40008C93A0E8B0E0E0E8F0E080818E7F8C939A
:101A500020C089818A3079F4A0E8B0E0E0E8F0E0C5
:101A6000808182608C93A0E8B0E0E0E8F0E08081C3
:101A700081608C930EC0A0E8B0E0E0E8F0E08081E7
:101A80008D7F8C93A0E8B0E0E0E8F0E08081816099
:101A90008C93E8E8F0E011821082EAE8F0E011822D
:101AA00010820F90CF91DF910895DF93CF9300D0F4
:101AB000CDB7DEB79A838983A0E8B0E0E0E8F0E034
:101AC00080818E7F8C93A0E8B0E0E0E8F0E0808138
:101AD00082608C93A1E8B0E0E1E8F0E0808188606A
:101AE0008C93A1E8B0E0E1E8F0E0808180618C9324
:101AF000E6E8F0E089819A8191838083E8E8F0E06C
:101B000011821082EAE8F0E0118210820F900F90AB
:101B1000CF91DF910895DF93CF93CDB7DEB7A0E8E3
:101B2000B0E0E0E8F0E080818D7F8C93A0E8B0E049
:101B3000E0E8F0E080818E7F8C930E94CE0D0E94C1
:101B4000E30DCF91DF910895DF93CF93CDB7DEB74B
:101B5000A0E8B0E0E0E8F0E0808180688C93A0E845
:101B6000B0E0E0E8F0E080818F7B8C93CF91DF9153
:101B70000895DF93CF93CDB7DEB7A0E8B0E0E0E8FB
:101B8000F0E0808180628C93A0E8B0E0E0E8F0E0D3
:101B900080818F7E8C93CF91DF910895DF93CF93D7
:101BA000CDB7DEB7A0E8B0E0E0E8F0E080818F7765
:101BB0008C93A0E8B0E0E0E8F0E080818F7B8C932C
:101BC000CF91DF910895DF93CF93CDB7DEB7A0E833
:101BD000B0E0E0E8F0E080818F7D8C93A0E8B0E099
:101BE000E0E8F0E080818F7E8C93CF91DF910895C3
:101BF000DF93CF9300D0CDB7DEB79A838983E8E82F
:101C0000F0E089819A81918380830F900F90CF912A
:101C1000DF910895DF93CF9300D0CDB7DEB79A83DD
:101C20008983EAE8F0E089819A81918380830F902B
:101C30000F90CF91DF9108951F920F920FB60F92E0
:101C400011242F933F934F935F936F937F938F93C1
:101C50009F93AF93BF93EF93FF93DF93CF93CDB752
:101C6000DEB78091430590914405A0914505B09160
:101C700046050196A11DB11D80934305909344052F
:101C8000A0934505B093460580914705909148057E
:101C9000A0914905B0914A050196A11DB11D8093FF
:101CA000470590934805A0934905B0934A05809154
:101CB000DE049091DF04009729F0E091DE04F091BA
:101CC000DF040995CF91DF91FF91EF91BF91AF9123
:101CD0009F918F917F916F915F914F913F912F9144
:101CE0000F900FBE0F901F9018951F920F920FB676
:101CF0000F9211242F933F934F935F936F937F9392
:101D00008F939F93AF93BF93EF93FF93DF93CF9303
:101D1000CDB7DEB78091E0049091E104009729F0FF
:101D2000E091E004F091E1040995CF91DF91FF91FA
:101D3000EF91BF91AF919F918F917F916F915F9143
:101D40004F913F912F910F900FBE0F901F901895BC
:101D50001F920F920FB60F9211242F933F934F9320
:101D60005F936F937F938F939F93AF93BF93EF9303
:101D7000FF93DF93CF93CDB7DEB780914B05909162
:101D80004C05A0914D05B0914E050196A11DB11DC8
:101D900080934B0590934C05A0934D05B0934E0551
:101DA0008091E8049091E904009729F0E091E8041B
:101DB000F091E9040995CF91DF91FF91EF91BF91E7
:101DC000AF919F918F917F916F915F914F913F91D3
:101DD0002F910F900FBE0F901F9018951F920F928A
:101DE0000FB60F9211242F933F934F935F936F93EE
:101DF0007F938F939F93AF93BF93EF93FF93DF9363
:101E0000CF93CDB7DEB78091E2049091E3040097C1
:101E100029F0E091E204F091E3040995CF91DF917C
:101E2000FF91EF91BF91AF919F918F917F916F91B2
:101E30005F914F913F912F910F900FBE0F901F9088
:101E400018951F920F920FB60F9211242F933F9364
:101E50004F935F936F937F938F939F93AF93BF93B2
:101E6000EF93FF93DF93CF93CDB7DEB78091E40478
:101E70009091E504009729F0E091E404F091E504E5
:101E80000995CF91DF91FF91EF91BF91AF919F9114
:101E90008F917F916F915F914F913F912F910F9013
:101EA0000FBE0F901F9018951F920F920FB60F92B2
:101EB00011242F933F934F935F936F937F938F934F
:101EC0009F93AF93BF93EF93FF93DF93CF93CDB7E0
:101ED000DEB78091E6049091E704009729F0E09145
:101EE000E604F091E7040995CF91DF91FF91EF911E
:101EF000BF91AF919F918F917F916F915F914F9122
:101F00003F912F910F900FBE0F901F9018951F9229
:101F10000F920FB60F9211242F933F934F935F931D
:101F20006F937F938F939F93AF93BF93EF93FF93A1
:101F3000DF93CF93CDB7DEB78091EA049091EB04A5
:101F4000009729F0E091EA04F091EB040995CF9114
:101F5000DF91FF91EF91BF91AF919F918F917F9111
:101F60006F915F914F913F912F910F900FBE0F9006
:101F70001F9018951F920F920FB60F9211242F9356
:101F80003F934F935F936F937F938F939F93AF9301
:101F9000BF93EF93FF93DF93CF93CDB7DEB78091DD
:101FA000EA049091EB04009729F0E091EA04F091A3
:101FB000EB040995CF91DF91FF91EF91BF91AF9124
:101FC0009F918F917F916F915F914F913F912F9151
:101FD0000F900FBE0F901F901895DF93CF9300D0F6
:101FE000CDB7DEB79A83898389819A819093ED0476
:101FF0008093EC040F900F90CF91DF910895DF93C1
:10200000CF930F92CDB7DEB7898389818A3031F4BF
:10201000E091EC04F091ED048DE00995E091EC0481
:10202000F091ED04898109950F90CF91DF9108958A
:10203000DF93CF9300D0CDB7DEB79A8389838981B0
:102040009A81009789F00BC0E981FA81208189810A
:102050009A8101969A838983822F0E94FF0FE981DA
:10206000FA818081882381F70F900F90CF91DF91C3
:102070000895DF93CF93CDB7DEB72A970FB6F894C4
:10208000DEBF0FBECDBF9A8389837C836B835E8363
:102090004D8318861F8289819A81009709F449C06F
:1020A0002F81388519868B819C812817390710F478
:1020B00081E089878F819885019698878F8381E059
:1020C00099858927882391F4E981FA8180818A871B
:1020D0008A85882311F091E09A878A8529813A813F
:1020E0002F5F3F4F3A8329838823D1F618861F82BA
:1020F00019C0E981FA818081882361F0E981FA8140
:10210000208189819A8101969A838983822F0E94F6
:10211000FF0F03C080E20E94FF0F8F819885019618
:1021200098878F832F8138858D819E812817390765
:1021300000F32A960FB6F894DEBF0FBECDBFCF9145
:10214000DF910895DF93CF9300D000D000D0CDB7BA
:10215000DEB79D838C838C819D810097B1F003C095
:102160008E810E94FF0F8C819D819B838A838C814D
:102170009D8101969D838C83EA81FB818491898373
:1021800089818E838E81882359F726960FB6F8941D
:10219000DEBF0FBECDBFCF91DF910895DF93CF9308
:1021A000CDB7DEB78AE00E94FF0FCF91DF9108958F
:1021B000DF93CF9300D000D0CDB7DEB78C838C8176
:1021C000882F90E08F70907080509F4F9B838A8300
:1021D000EA81FB818491898389810E94FF0F0F909E
:1021E0000F900F900F90CF91DF910895DF93CF93D1
:1021F0000F92CDB7DEB78983898182958F700E9457
:10220000D81089810E94D8100F90CF91DF91089546
:10221000DF93CF9300D0CDB7DEB79A8389838981CE
:102220009A81892F99270E94F61089810E94F610C1
:102230000F900F90CF91DF910895DF93CF9300D04F
:1022400000D0CDB7DEB769837A838B839C83898185
:102250009A81AB81BC81CD01AA27BB270E940811BE
:1022600089819A810E9408110F900F900F900F9012
:10227000CF91DF910895EF92FF920F931F93DF9319
:10228000CF93CDB7DEB7E8970FB6F894DEBF0FBE99
:10229000CDBF8EA76FA748AB29ABEAAAFBAA0CABB0
:1022A0001DAB88A98823B1F08AA99BA9ACA9BDA9B7
:1022B000BB2384F48AA99BA9ACA9BDA9B095A0951C
:1022C000909581959F4FAF4FBF4F88879987AA8779
:1022D000BB8708C08AA99BA9ACA9BDA98887998793
:1022E000AA87BB8788A98EAB8EA9882311F081E0CD
:1022F0008EAB9EA98FA5891B81508F83CE010E9630
:1023000080969D878C878C859D8501979D878C877E
:10231000EC85FD8510828C859D8501979D878C8736
:102320008EA5282F30E040E050E088859985AA8569
:10233000BB85BC01CD010E94841DDC01CB018F70E7
:10234000907080509F4F9E838D83ED81FE8184919C
:102350008C838C81EC85FD8580838EA5282F30E0D1
:1023600040E050E088859985AA85BB85BC01CD01F8
:102370000E94841DDA01C90188879987AA87BB87D3
:1023800047C088859985AA85BB850097A105B105B9
:10239000B1F18C859D8501979D878C878EA5282F0F
:1023A00030E040E050E088859985AA85BB85BC0176
:1023B000CD010E94841DDC01CB018F709070805094
:1023C0009F4F9B838A83EA81FB81849189838981E2
:1023D000EC85FD8580838EA5282F30E040E050E01D
:1023E00088859985AA85BB85BC01CD010E94841D85
:1023F000DA01C90188879987AA87BB8709C08C85BC
:102400009D8501979D878C87EC85FD8589A98083B3
:102410008F818FAB8FA9882311F081E08FAB8FA9BB
:102420009F8191509F83882309F0ABCF88A988238F
:1024300061F18AA99BA9ACA9BDA9BB2354F48C85E1
:102440009D8501979D878C87EC85FD858DE2808336
:102450001CC08AA99BA9ACA9BDA9181619061A0601
:102460001B0654F48C859D8501979D878C87EC8590
:10247000FD858BE2808309C08C859D8501979D87B2
:102480008C87EC85FD8580E280838FA58F830BC0D0
:10249000EC85FD8520818C859D8501969D878C87A7
:1024A000822F0E94FF0F8F8188AF88AD882311F0A3
:1024B00081E088AF88AD9F8191509F83882341F749
:1024C000E8960FB6F894DEBF0FBECDBFCF91DF9177
:1024D0001F910F91FF90EF900895DF93CF93CDB7A9
:1024E000DEB763970FB6F894DEBF0FBECDBFCE0147
:1024F0004B969F878E8711C08D85882359F480E085
:1025000090E063960FB6F894DEBF0FBECDBFCF91BB
:10251000DF9108958D850E94FF0F888D882381F0BB
:10252000898D9A8D9E838D83898D9A8D01969A8F40
:10253000898FED81FE8184918C838C818B8B09C086
:10254000E98DFA8D20812B8B898D9A8D01969A8F3A
:10255000898F3B893D878D85853271F6888D8823EB
:1025600081F0898D9A8D9B838A83898D9A8D0196BE
:102570009A8F898FEA81FB818491898389818A8BF3
:1025800009C0E98DFA8D80818A8B898D9A8D01969B
:102590009A8F898F9A899D878D85282F30E0398B76
:1025A000288B8889998984369105C1F028893989D1
:1025B00028373105E1F0888999898336910551F4EE
:1025C0002E853F85C90102969F878E87F9018081FC
:1025D00091818D878D850E94FF0F9FCF8AE090E0CB
:1025E00098878F8380E197E29A87898708C080E186
:1025F00090E098878F8380E090E19A8789872E8585
:102600003F85C90102969F878E87F901808191815C
:102610009C878B878D85843629F58B859C859923AE
:10262000ACF48B859C85909581959F4F9C878B877B
:102630008DE20E94FF0F0AC089859A852AE030E06A
:10264000B9010E945D1DCB019A87898789859A858A
:102650008230910538F029853A858B859C858217D3
:10266000930750F38B859C8529853A85B9010E9493
:102670005D1DCB010E94D8108B859C8529853A85EC
:10268000B9010E945D1D9C878B8789859A852F8162
:102690003885B9010E945D1DCB019A87898789859C
:1026A0009A850097F9F639CFDF93CF93CDB7DEB790
:1026B000E0E3F0E01082E1E3F0E01082E7E0F1E037
:1026C0001082E8E0F1E01082E1E2F0E08FEF808339
:1026D000E4E2F0E080E48083E7E2F0E08FEF8083E3
:1026E000EAE2F0E08BEF8083EDE2F0E08EEF8083B2
:1026F000A4E3B0E0E4E3F0E0808180628C93A3E3A4
:10270000B0E0E3E3F0E080818F7D8C93E1E0F1E0E5
:102710008EEF8083E4E0F1E08EEF8083CF91DF9154
:102720000895DF93CF9300D000D0CDB7DEB7698393
:102730007A838B839C830BC089819A81AB81BC8116
:102740000197A109B10989839A83AB83BC838981ED
:102750009A81AB81BC810097A105B10569F70F9003
:102760000F900F900F90CF91DF910895DF93CF934B
:10277000CDB7DEB7A5E2B0E0E5E2F0E080818064AD
:102780008C93CF91DF910895DF93CF93CDB7DEB7D0
:10279000A5E2B0E0E5E2F0E080818F7B8C93CF9101
:1027A000DF910895DF93CF93CDB7DEB7E6E4F0E095
:1027B00010820E94D10CCF91DF910895DF93CF93C7
:1027C00000D0CDB7DEB7E2E3F0E08081882F90E063
:1027D000807290701A821982009721F481E090E053
:1027E0009A83898389819A810F900F90CF91DF918D
:1027F0000895DF93CF9300D000D000D0CDB7DEB7DF
:1028000069837A838B839C8389819A81AB81BC8124
:10281000BB23C4F089819A81AB81BC8125E030E083
:1028200040E050E0BC01CD010E94A61DDA01C901C3
:10283000880F991FFC01E050FE4F208131813E83BB
:102840002D832CC089819A81AB81BC81B095A095E4
:10285000909581959F4FAF4FBF4F25E030E040E00E
:1028600050E0BC01CD010E94A61DDA01C9019C0106
:10287000AD0188E490E0A0E0B0E0821B930BA40BD4
:10288000B50B880F991FFC01E050FE4F80819181AC
:1028900022273327281B390B3E832D838D819E8170
:1028A00026960FB6F894DEBF0FBECDBFCF91DF9155
:1028B0000895DF93CF9300D000D000D0CDB7DEB71E
:1028C00069837A838B839C8389819A81AB81BC8164
:1028D0008A559040A040B04089839A83AB83BC83E3
:1028E00089819A81AB81BC81BB23C4F089819A81A3
:1028F000AB81BC8125E030E040E050E0BC01CD017F
:102900000E94A61DDA01C901880F991FFC01E05041
:10291000FE4F208131813E832D832CC089819A8195
:10292000AB81BC81B095A095909581959F4FAF4F9D
:10293000BF4F25E030E040E050E0BC01CD010E94F7
:10294000A61DDA01C9019C01AD0188E490E0A0E078
:10295000B0E0821B930BA40BB50B880F991FFC01F1
:10296000E050FE4F8081918122273327281B390BAD
:102970003E832D838D819E8126960FB6F894DEBF0F
:102980000FBECDBFCF91DF9108950F931F93DF93BB
:10299000CF9300D000D000D0CDB7DEB769837A8363
:1029A0008B839C8389819A81AB81BC818A35910517
:1029B000A105B10521F189819A81AB81BC81863A5B
:1029C0002FEF92072FEFA2072FEFB207C1F08981F7
:1029D0009A81AB81BC818E3041E0940740E0A4072E
:1029E00040E0B40761F089819A81AB81BC81823F6C
:1029F0005EEF95075FEFA5075FEFB50719F41E823D
:102A00001D8224C089819A81AB81BC81BC01CD012A
:102A10000E9459148C0189819A81AB81BC81BC01CF
:102A2000CD010E94F9139C01C801B9010E94711DDA
:102A3000CB019C01220F331FC901880F991F880FFA
:102A4000991FA901480F591F5E834D838D819E8177
:102A500026960FB6F894DEBF0FBECDBFCF91DF91A3
:102A60001F910F910895DF93CF93CDB7DEB72A97CB
:102A70000FB6F894DEBF0FBECDBF84EF91E0A0E0AB
:102A8000B0E08F839887A987BA8784EF91E0A0E0B0
:102A9000B0E08B839C83AD83BE8388E090E09A8313
:102AA00089830E9440162091920230919302809176
:102AB0009402909195028217930788F420919202D4
:102AC000309193028091940290919502A901481B44
:102AD000590BCA019093F1048093F00410C0209127
:102AE0009402309195028091920290919302A901F3
:102AF000481B590BCA019093EF048093EE040E9487
:102B0000401620919202309193028091940290910C
:102B100095028217930700F520919202309193025B
:102B20008091940290919502281B390B89819A819A
:102B30008217930788F486E292E0A0E0B0E08F83EA
:102B40009887A987BA8786E292E0A0E0B0E08B83FD
:102B50009C83AD83BE833BC020919402309195024B
:102B600080919202909193028217930700F5209131
:102B70009402309195028091920290919302281BC9
:102B8000390B89819A818217930788F482E593E053
:102B9000A0E0B0E08F839887A987BA8782E593E0A9
:102BA000A0E0B0E08B839C83AD83BE8310C088E53A
:102BB00092E0A0E0B0E08F839887A987BA8780E28F
:102BC00093E0A0E0B0E08B839C83AD83BE83209133
:102BD000940230919502409192025091930261E1EA
:102BE00071E08B819C81AD81BE81BF93AF939F9338
:102BF0008F933F932F938F819885A985BA85BF9333
:102C0000AF939F938F935F934F937F936F9381E0E5
:102C10008F930E946D128DB79EB70F960FB6F894E2
:102C20009EBF0FBE8DBFAEE2B0E0EEE2F0E080816D
:102C300080648C938F819885A985BA85BC01CD016C
:102C40000E949113AEE2B0E0EEE2F0E080818F7B73
:102C50008C93A8E2B0E0E8E2F0E0808180688C9399
:102C60008B819C81AD81BE81BC01CD010E949113FD
:102C7000A8E2B0E0E8E2F0E080818F778C933FCF6C
:102C8000DF93CF93CDB7DEB782E00E940D02282FED
:102C900030E08091F0049091F104820F931F9093A3
:102CA0009502809394028EE00E940D02282F30E05E
:102CB0008091EE049091EF04820F931F9093930202
:102CC00080939202CF91DF910895DF93CF93CDB798
:102CD000DEB70E94C4130E94DE13009711F00E9419
:102CE000B613E0E3F0E08FEF8083E7E0F1E08FEFF1
:102CF0008083A2E0B1E0E2E0F1E0808180648C9327
:102D0000A2E0B1E0E2E0F1E0808180628C93A2E099
:102D1000B1E0E2E0F1E0808180618C93A2E0B1E07B
:102D2000E2E0F1E0808188608C93A2E0B1E0E2E033
:102D3000F1E0808184608C93AEE2B0E0EEE2F0E0FE
:102D4000808180688C93AEE2B0E0EEE2F0E08081BA
:102D500080648C93AEE2B0E0EEE2F0E080818062CD
:102D60008C93AEE2B0E0EEE2F0E0808180618C9383
:102D7000AEE2B0E0EEE2F0E0808188608C93AEE2FB
:102D8000B0E0EEE2F0E0808184608C93A8E2B0E0F5
:102D9000E8E2F0E0808181608C93A8E2B0E0E8E2B4
:102DA000F0E0808182608C93A8E2B0E0E8E2F0E09D
:102DB000808184608C93A8E2B0E0E8E2F0E080815A
:102DC00088608C93A8E2B0E0E8E2F0E08081806166
:102DD0008C93A8E2B0E0E8E2F0E0808180628C931E
:102DE000A8E2B0E0E8E2F0E0808180648C93A8E2A1
:102DF000B0E0E8E2F0E0808180688C93A5E0B1E08B
:102E0000E5E0F1E0808180648C93A2E2B0E0E2E250
:102E1000F0E0808180688C93A2E2B0E0E2E2F0E032
:102E2000808180648C93A2E2B0E0E2E2F0E08081F5
:102E300080628C93A2E2B0E0E2E2F0E08081806107
:102E40008C93A2E2B0E0E2E2F0E0808188608C93B3
:102E5000A2E2B0E0E2E2F0E0808184608C93A2E242
:102E6000B0E0E2E2F0E0808182608C93A2E2B0E028
:102E7000E2E2F0E0808181608C93A1E3B0E0E1E3E5
:102E8000F0E0808181608C93A1E3B0E0E1E3F0E0C9
:102E9000808182608C93A1E3B0E0E1E3F0E0808187
:102EA00084608C93A1E3B0E0E1E3F0E0808188608E
:102EB0008C93A1E3B0E0E1E3F0E0808180618C934A
:102EC000A1E3B0E0E1E3F0E0808180628C93A1E3D4
:102ED000B0E0E1E3F0E0808180648C93A1E3B0E0B6
:102EE000E1E3F0E0808180688C93A8E0B1E0E8E065
:102EF000F1E0808181608C93A8E0B1E0E8E0F1E04E
:102F0000808182608C93A8E0B1E0E8E0F1E080810C
:102F100084608C93A8E0B1E0E8E0F1E08081886013
:102F20008C93A8E0B1E0E8E0F1E0808180618C93CF
:102F3000A8E0B1E0E8E0F1E0808180628C93A8E055
:102F4000B1E0E8E0F1E0808180648C93A8E0B1E03A
:102F5000E8E0F1E0808180688C9380E293E00E9459
:102F6000FB0B82E296E00E94ED0F89E691E09F93D1
:102F70008F9381E08F930E946D120F900F900F90AE
:102F800080E396E00E94ED0F86E691E09F938F9399
:102F900081E08F930E946D120F900F900F908EE33F
:102FA00096E00E94ED0F83E691E09F938F9381E07E
:102FB0008F930E946D120F900F900F908CE496E00B
:102FC0000E94ED0F80E691E09F938F9381E08F93B5
:102FD0000E946D120F900F900F90A2E0B1E0E2E01E
:102FE000F1E080818F7B8C93A2E0B1E0E2E0F1E040
:102FF00080818F7D8C93A2E0B1E0E2E0F1E08081FE
:103000008F7E8C93A2E0B1E0E2E0F1E08081877FE7
:103010008C93A2E0B1E0E2E0F1E080818B7F8C93C1
:10302000AEE2B0E0EEE2F0E080818F778C93AEE22A
:10303000B0E0EEE2F0E080818F7B8C93AEE2B0E016
:10304000EEE2F0E080818F7D8C93AEE2B0E0EEE2C4
:10305000F0E080818F7E8C93AEE2B0E0EEE2F0E0B3
:103060008081877F8C93AEE2B0E0EEE2F0E0808179
:103070008B7F8C93A8E2B0E0E8E2F0E080818E7F65
:103080008C93A8E2B0E0E8E2F0E080818D7F8C9341
:10309000A8E2B0E0E8E2F0E080818B7F8C93A8E2C8
:1030A000B0E0E8E2F0E08081877F8C93A8E2B0E0B6
:1030B000E8E2F0E080818F7E8C93A8E2B0E0E8E265
:1030C000F0E080818F7D8C93A8E2B0E0E8E2F0E050
:1030D00080818F7B8C93A8E2B0E0E8E2F0E0808111
:1030E0008F778C93A5E0B1E0E5E0F1E080818F7B04
:1030F0008C93A2E2B0E0E2E2F0E080818F778C93E3
:10310000A2E2B0E0E2E2F0E080818F7B8C93A2E269
:10311000B0E0E2E2F0E080818F7D8C93A2E2B0E04B
:10312000E2E2F0E080818F7E8C93A2E2B0E0E2E206
:10313000F0E08081877F8C93A2E2B0E0E2E2F0E0F1
:1031400080818B7F8C93A2E2B0E0E2E2F0E08081AC
:103150008D7F8C93A2E2B0E0E2E2F0E080818E7F8E
:103160008C93A1E3B0E0E1E3F0E080818E7F8C936B
:10317000A1E3B0E0E1E3F0E080818D7F8C93A1E3F7
:10318000B0E0E1E3F0E080818B7F8C93A1E3B0E0DD
:10319000E1E3F0E08081877F8C93A1E3B0E0E1E39D
:1031A000F0E080818F7E8C93A1E3B0E0E1E3F0E07A
:1031B00080818F7D8C93A1E3B0E0E1E3F0E080813A
:1031C0008F7B8C93A1E3B0E0E1E3F0E080818F7727
:1031D0008C93A8E0B1E0E8E0F1E080818E7F8C93F1
:1031E000A8E0B1E0E8E0F1E080818D7F8C93A8E079
:1031F000B1E0E8E0F1E080818B7F8C93A8E0B1E062
:10320000E8E0F1E08081877F8C93A8E0B1E0E8E01E
:10321000F1E080818F7E8C93A8E0B1E0E8E0F1E0FE
:1032200080818F7D8C93A8E0B1E0E8E0F1E08081BF
:103230008F7B8C93A8E0B1E0E8E0F1E080818F77AC
:103240008C9380E293E00E94FB0B82E296E00E9466
:10325000ED0F8AE591E09F938F9381E08F930E9419
:103260006D120F900F900F9080E396E00E94ED0F8B
:1032700084E591E09F938F9381E08F930E946D127C
:103280000F900F900F908EE396E00E94ED0F8EE46A
:1032900091E09F938F9381E08F930E946D120F9026
:1032A0000F900F908CE496E00E94ED0F88E491E07F
:1032B0009F938F9381E08F930E946D120F900F90D8
:1032C0000F906CED7FEF80E090E00E949113CF9122
:1032D000DF910895DF93CF93CDB7DEB7A0970FB6F8
:1032E000F894DEBF0FBECDBF0E94C4130E94DE1350
:1032F000009711F00E94B613A8E2B0E0E8E2F0E017
:10330000808181608C9368E671E080E090E00E94AB
:103310009113A8E2B0E0E8E2F0E080818E7F8C9328
:10332000A8E2B0E0E8E2F0E0808182608C9368E699
:1033300071E080E090E00E949113A8E2B0E0E8E242
:10334000F0E080818D7F8C93A8E2B0E0E8E2F0E0CD
:10335000808184608C9368E671E080E090E00E9458
:103360009113A8E2B0E0E8E2F0E080818B7F8C93DB
:10337000A8E2B0E0E8E2F0E0808188608C9368E643
:1033800071E080E090E00E949113A8E2B0E0E8E2F2
:10339000F0E08081877F8C93A8E2B0E0E8E2F0E083
:1033A000808180618C9368E671E080E090E00E940B
:1033B0009113A8E2B0E0E8E2F0E080818F7E8C9388
:1033C000A8E2B0E0E8E2F0E0808180628C9368E6F9
:1033D00071E080E090E00E949113A8E2B0E0E8E2A2
:1033E000F0E080818F7D8C93A8E2B0E0E8E2F0E02D
:1033F000808180648C9368E671E080E090E00E94B8
:103400009113A8E2B0E0E8E2F0E080818F7B8C933A
:10341000A8E2B0E0E8E2F0E0808180688C9368E6A2
:1034200071E080E090E00E949113A8E2B0E0E8E251
:10343000F0E080818F778C93A5E0B1E0E5E0F1E0EA
:10344000808180648C9368E671E080E090E00E9467
:103450009113A5E0B1E0E5E0F1E080818F7B8C93F2
:10346000A2E2B0E0E2E2F0E0808181608C9368E665
:1034700071E080E090E00E949113A2E2B0E0E2E20D
:10348000F0E080818E7F8C93A2E2B0E0E2E2F0E097
:10349000808182608C9368E671E080E090E00E9419
:1034A0009113A2E2B0E0E2E2F0E080818D7F8C93A4
:1034B000A2E2B0E0E2E2F0E0808184608C9368E612
:1034C00071E080E090E00E949113A2E2B0E0E2E2BD
:1034D000F0E080818B7F8C93A2E2B0E0E2E2F0E04A
:1034E000808188608C9368E671E080E090E00E94C3
:1034F0009113A2E2B0E0E2E2F0E08081877F8C935A
:10350000A2E2B0E0E2E2F0E0808180618C9368E6C4
:1035100071E080E090E00E949113A2E2B0E0E2E26C
:10352000F0E080818F7E8C93A2E2B0E0E2E2F0E0F6
:10353000808180628C9368E671E080E090E00E9478
:103540009113A2E2B0E0E2E2F0E080818F7D8C9303
:10355000A2E2B0E0E2E2F0E0808180648C9368E671
:1035600071E080E090E00E949113A2E2B0E0E2E21C
:10357000F0E080818F7B8C93A2E2B0E0E2E2F0E0A9
:10358000808180688C9368E671E080E090E00E9422
:103590009113A2E2B0E0E2E2F0E080818F778C93B9
:1035A000AEE2B0E0EEE2F0E0808184608C9368E609
:1035B00071E080E090E00E949113AEE2B0E0EEE2B4
:1035C000F0E080818B7F8C93AEE2B0E0EEE2F0E041
:1035D000808188608C9368E671E080E090E00E94D2
:1035E0009113AEE2B0E0EEE2F0E08081877F8C9351
:1035F000AEE2B0E0EEE2F0E0808180618C9368E6BC
:1036000071E080E090E00E949113AEE2B0E0EEE263
:10361000F0E080818F7E8C93AEE2B0E0EEE2F0E0ED
:10362000808180628C9368E671E080E090E00E9487
:103630009113AEE2B0E0EEE2F0E080818F7D8C93FA
:10364000AEE2B0E0EEE2F0E0808180648C9368E668
:1036500071E080E090E00E949113AEE2B0E0EEE213
:10366000F0E080818F7B8C93AEE2B0E0EEE2F0E0A0
:10367000808180688C9368E671E080E090E00E9431
:103680009113AEE2B0E0EEE2F0E080818F778C93B0
:10369000A2E0B1E0E2E0F1E0808184608C9368E632
:1036A00071E080E090E00E949113A2E0B1E0E2E0DE
:1036B000F1E080818B7F8C93A2E0B1E0E2E0F1E069
:1036C000808188608C9368E671E080E090E00E94E1
:1036D0009113A2E0B1E0E2E0F1E08081877F8C937A
:1036E000A2E0B1E0E2E0F1E0808180618C9368E6E5
:1036F00071E080E090E00E949113A2E0B1E0E2E08E
:10370000F1E080818F7E8C93A2E0B1E0E2E0F1E015
:10371000808180628C9368E671E080E090E00E9496
:103720009113A2E0B1E0E2E0F1E080818F7D8C9323
:10373000A2E0B1E0E2E0F1E0808180648C9368E691
:1037400071E080E090E00E949113A2E0B1E0E2E03D
:10375000F1E080818F7B8C9380E00E940D02882FA6
:1037600090E098A38F8F81E00E940D02882F90E057
:103770009E8F8D8F82E00E940D02882F90E09C8F9B
:103780008B8F83E00E940D02882F90E09A8F898FA3
:1037900084E00E940D02882F90E0988F8F8B85E047
:1037A0000E940D02882F90E09E8B8D8B86E00E94F8
:1037B0000D02882F90E09C8B8B8B87E00E940D027E
:1037C000882F90E09A8B898B88E00E940D02882FC9
:1037D00090E0988B8F8789E00E940D02882F90E0FF
:1037E0009E878D878AE00E940D02882F90E09C873B
:1037F0008B878BE00E940D02882F90E09A87898743
:103800008CE00E940D02882F90E098878F838DE0D6
:103810000E940D02882F90E09E838D838EE00E948F
:103820000D02882F90E09C838B838FE00E940D0215
:10383000882F90E09A83898380E396E00E94ED0FC1
:1038400026EA31E089899A899F938F938B899C8995
:103850009F938F938D899E899F938F938F89988D46
:103860009F938F93898D9A8D9F938F938B8D9C8D32
:103870009F938F938D8D9E8D9F938F938F8D98A106
:103880009F938F933F932F9381E08F930E946D12AC
:103890008DB79EB743960FB6F8949EBF0FBE8DBFEF
:1038A00025E731E089819A819F938F938B819C8159
:1038B0009F938F938D819E819F938F938F81988506
:1038C0009F938F9389859A859F938F938B859C85F2
:1038D0009F938F938D859E859F938F938F859889D6
:1038E0009F938F933F932F9381E08F930E946D124C
:1038F0008DB79EB743960FB6F8949EBF0FBE8DBF8F
:1039000082E296E00E94ED0F82E791E09F938F9311
:1039100081E08F930E946D120F900F900F908EE3B5
:1039200096E00E94ED0F8FE691E09F938F9381E0E8
:103930008F930E946D120F900F900F908CE496E081
:103940000E94ED0F8CE691E09F938F9381E08F931F
:103950000E946D120F900F900F906CED7FEF80E042
:1039600090E00E949113A0960FB6F894DEBF0FBEB0
:10397000CDBFCF91DF910895DF93CF9300D000D0DA
:10398000CDB7DEB71C821B821A8219820E94F70310
:1039900040E056E960E070E080E00E94180540E0F9
:1039A00052EC61E070E081E00E94180540E056E9C9
:1039B00060E070E082E00E94180540E056E960E0B7
:1039C00070E083E00E94180580E396E00E94ED0F0E
:1039D0000E94DA0A0E9454130E94200185E00E948E
:1039E000610181E00E9475010E94C4138EEE91E096
:1039F0009F938F9381E08F930E946D120F900F9091
:103A00000F901C821B8216C068E873E180E090E092
:103A10000E9491138CEE91E09F938F9381E08F939E
:103A20000E946D120F900F900F908B819C810196D8
:103A30009C838B838B819C81813191052CF360E782
:103A400077E180E090E00E9491131C821B820CC001
:103A50008B810E940D02882F90E09A8389838B814D
:103A60009C8101969C838B838B819C818031910505
:103A70007CF30E94B6130E946516FDCF629FD001B1
:103A8000739FF001829FE00DF11D649FE00DF11D19
:103A9000929FF00D839FF00D749FF00D659FF00DC8
:103AA0009927729FB00DE11DF91F639FB00DE11DB5
:103AB000F91FBD01CF0111240895AA1BBB1B51E1C1
:103AC00007C0AA1FBB1FA617B70710F0A61BB70B8E
:103AD000881F991F5A95A9F780959095BC01CD0133
:103AE000089597FB092E07260AD077FD04D0E5DF5D
:103AF00006D000201AF4709561957F4F0895F6F76F
:103B0000909581959F4F0895A1E21A2EAA1BBB1B89
:103B1000FD010DC0AA1FBB1FEE1FFF1FA217B30799
:103B2000E407F50720F0A21BB30BE40BF50B661FAF
:103B3000771F881F991F1A9469F760957095809573
:103B400090959B01AC01BD01CF01089597FB092E13
:103B500005260ED057FD04D0D7DF0AD0001C38F45C
:103B600050954095309521953F4F4F4F5F4F0895A9
:103B7000F6F790958095709561957F4F8F4F9F4F89
:063B80000895F894FFCF48
:103B860064006400620061005E005B005700520042
:103B96004D0047004000390032002A0022001A007A
:103BA600110009000000F7FFEFFFE6FFDEFFD6FF7A
:103BB600CEFFC7FFC0FFB9FFB3FFAEFFA9FFA5FF4A
:103BC600A2FF9FFF9EFF9CFF9CFF9CFF9EFF9FFF07
:103BD600A2FFA5FFA9FFAEFFB3FFB9FFC0FFC7FF56
:103BE600CEFFD6FFDEFFE6FFEFFFF7FF000009007E
:103BF60011001A0022002A00320039004000470056
:103C06004D00520057005B005E00610062006400D8
:063C160064008000800044
:00000001FF
